:020000040000FA
:020000006D2869
:08000800A200030EA3000B117E
:10001000A00F0B28A10A230E8300A20E220E0900B6
:1000200036308A010F39820787288A288D28902840
:100030009528A028AA28AF28EE28EE28EE28EE283A
:10004000EE28EE28EE28EE288A010F3982072034A8
:100050001834183420341D34193419341E3419342A
:100060001B341B3420341B3419341D3420348A01D2
:100070000F39820720341D341934163414341334E4
:100080001134103410341134133414341634193438
:100090001D3420348A011F39820720341E341D3458
:1000A0001C341B341A34193418341A3419341B34E0
:1000B00019341A34193418341834193418341934DA
:1000C0001A341B3419341A341B341A341B341C34BC
:1000D0001D341C341D341E341F348316FE3085003D
:1000E0000F3086008E1508308100831207309F0084
:1000F000850186018101A001A101A701A0308B002B
:1001000080308600A001A9010608FF3A11280030BE
:10011000A40092281830A40092281030A40092283D
:100120000830A4001F30AA00BA282708A800A80C8D
:10013000A80CA80C1F30AA0028084A20A400BA283E
:100140002708A800A80CA80C1F30AA002808242003
:10015000A400BA282708A800A80CA80CB4282708CF
:10016000A800A80CA80CA80C1F30AA00280837204B
:10017000A400BA2820082A05A500031DC628A9182E
:10018000CD28A91480308600A70ACD28A9102508FB
:100190002406031DCD28003086008518D528D028D8
:1001A000D1288518D528A1012914291C84282108C3
:1001B0007F3A031D8428003086008518DD28E0285A
:1001C000E1288518DD28851CE328E628E728E828AB
:1001D000E928851CE328EC28ED288028803086005B
:0E01E0008428AD002106031908002D08F2281E
:02400E00703F01
:00000001FF
